 gles1test1

 Timestamp is 4be8c3fd (Tue May 11 11:42:05 2010)

 Preferred load address is 00010000

 Start         Length     Name                   Class
 0001:00000000 00000004H .CRT$XCA                CODE
 0001:00000004 00000004H .CRT$XCZ                CODE
 0001:00000008 00000004H .CRT$XIA                CODE
 0001:0000000c 00000004H .CRT$XIZ                CODE
 0001:00000010 00000004H .CRT$XPA                CODE
 0001:00000014 00000004H .CRT$XPZ                CODE
 0001:00000018 00000004H .CRT$XTA                CODE
 0001:0000001c 00000004H .CRT$XTZ                CODE
 0001:00000020 00000370H .rdata                  CODE
 0001:00000390 00000027H .rdata$debug            CODE
 0001:000003b8 00000c98H .text                   CODE
 0001:00001050 00000014H .xdata                  CODE
 0001:00001064 00000028H .idata$2                CODE
 0001:0000108c 00000014H .idata$3                CODE
 0001:000010a0 000000d0H .idata$4                CODE
 0001:00001170 0000001cH .idata$6                CODE
 0001:0000118c 00000000H .edata                  CODE
 0002:00000000 000000d0H .idata$5                DATA
 0002:000000d0 000000d8H .data                   DATA
 0002:000001a8 0000401cH .bss                    DATA
 0003:00000000 00000070H .pdata                  DATA

  Address         Publics by Value              Rva+Base       Lib:Object

 0000:00000000       ___safe_se_handler_count   00000000     <absolute>
 0000:00000000       ___safe_se_handler_table   00000000     <absolute>
 0001:00000000       __xc_a                     00011000     corelib0:crt0init.obj
 0001:00000004       __xc_z                     00011004     corelib0:crt0init.obj
 0001:00000008       __xi_a                     00011008     corelib0:crt0init.obj
 0001:0000000c       __xi_z                     0001100c     corelib0:crt0init.obj
 0001:00000010       __xp_a                     00011010     corelib0:crt0init.obj
 0001:00000014       __xp_z                     00011014     corelib0:crt0init.obj
 0001:00000018       __xt_a                     00011018     corelib0:crt0init.obj
 0001:0000001c       __xt_z                     0001101c     corelib0:crt0init.obj
 0001:0000003c       ??_C@_0BA@ECMACICF@EGL_BAD_SURFACE?$AA@ 0001103c     gles1test1.obj
 0001:0000004c       ??_C@_0BC@OMABNJPB@EGL_BAD_PARAMETER?$AA@ 0001104c     gles1test1.obj
 0001:00000060       ??_C@_0BG@JCAPPMPM@EGL_BAD_NATIVE_WINDOW?$AA@ 00011060     gles1test1.obj
 0001:00000078       ??_C@_0BG@IANPFEBH@EGL_BAD_NATIVE_PIXMAP?$AA@ 00011078     gles1test1.obj
 0001:00000090       ??_C@_0O@GCFMIHO@EGL_BAD_MATCH?$AA@ 00011090     gles1test1.obj
 0001:000000a0       ??_C@_0BA@KHKFAGME@EGL_BAD_DISPLAY?$AA@ 000110a0     gles1test1.obj
 0001:000000b0       ??_C@_0BI@KBFIGPCO@EGL_BAD_CURRENT_SURFACE?$AA@ 000110b0     gles1test1.obj
 0001:000000c8       ??_C@_0BA@FPCJCEFK@EGL_BAD_CONTEXT?$AA@ 000110c8     gles1test1.obj
 0001:000000d8       ??_C@_0P@HOPKKPDK@EGL_BAD_CONFIG?$AA@ 000110d8     gles1test1.obj
 0001:000000e8       ??_C@_0BC@NLAJAPHP@EGL_BAD_ATTRIBUTE?$AA@ 000110e8     gles1test1.obj
 0001:000000fc       ??_C@_0O@PGDEJDGL@EGL_BAD_ALLOC?$AA@ 000110fc     gles1test1.obj
 0001:0000010c       ??_C@_0P@ELJNOEME@EGL_BAD_ACCESS?$AA@ 0001110c     gles1test1.obj
 0001:0000011c       ??_C@_0BE@JIJLFFAN@EGL_NOT_INITIALIZED?$AA@ 0001111c     gles1test1.obj
 0001:00000130       ??_C@_0M@JFIJMCIK@EGL_SUCCESS?$AA@ 00011130     gles1test1.obj
 0001:00000174       ??_C@_0CF@GLNKALBC@?8?$CFs?8?5returned?5egl?5error?5?8?$CFs?8?5?$CI0x@ 00011174     gles1test1.obj
 0001:0000019c       ??_C@_0DG@HMPOADHB@?9?9?9?9?9?9?9?9?9?9?9?9?9?9?9?9?9?9?9?9?9?5finished?5?9@ 0001119c     gles1test1.obj
 0001:000001d4       ??_C@_0P@PNPBPNLI@eglMakeCurrent?$AA@ 000111d4     gles1test1.obj
 0001:000001e4       ??_C@_0BB@KEKMNHDF@eglCreateContext?$AA@ 000111e4     gles1test1.obj
 0001:000001f8       ??_C@_0BH@MDMCFBDG@eglCreateWindowSurface?$AA@ 000111f8     gles1test1.obj
 0001:00000210       ??_C@_0BA@GKADIFMO@eglChooseConfig?$AA@ 00011210     gles1test1.obj
 0001:00000220       ??_C@_0O@OMNEJBKO@eglGetConfigs?$AA@ 00011220     gles1test1.obj
 0001:00000230       ??_C@_0O@EEJFKEKH@eglInitialize?$AA@ 00011230     gles1test1.obj
 0001:00000240       ??_C@_0DF@DFKFEDON@?9?9?9?9?9?9?9?9?9?9?9?9?9?9?9?9?9?9?9?9?9?5started?5?9?9@ 00011240     gles1test1.obj
 0001:00000278       ??_C@_1KE@BDGMONOJ@?$AAH?$AA?3?$AA?2?$AAW?$AAI?$AAN?$AAC?$AAE?$AA6?$AA0?$AA0?$AA?2?$AAP?$AAL?$AAA?$AAT?$AAF?$AAO?$AAR?$AAM?$AA?2?$AAS?$AAM?$AAD?$AAK?$AAV?$AA2?$AA1?$AA0?$AA?2?$AAS?$AAR@ 00011278     wince_unittests.obj
 0001:0000031c       ??_C@_1CI@OHCJFJPM@?$AAE?$AAR?$AAR?$AAO?$AAR?$AA?3?$AA?5?$AA?$CF?$AAs?$AA?5?$AAl?$AAi?$AAn?$AAe?$AA?5?$AA?$CF?$AAd?$AA?3?$AA?5?$AA?$AA@ 0001131c     wince_unittests.obj
 0001:00000344       ??_C@_1CK@MPGKAOE@?$AA?$CI?$AAe?$AAr?$AAr?$AAo?$AAr?$AA?5?$AAc?$AAo?$AAd?$AAe?$AA?3?$AA?5?$AA?$CF?$AAd?$AA?$CJ?$AA?3?$AA?5?$AA?$CF?$AAs?$AA?$AA@ 00011344     wince_unittests.obj
 0001:00000370       ??_C@_1M@DMCDIEDK@?$AAP?$AAK?$AAM?$AA1?$AA?3?$AA?$AA@ 00011370     wince_unittests.obj
 0001:0000037c       ??_C@_0L@GPAGIAIC@?9disablepm?$AA@ 0001137c     wince_unittests.obj
 0001:00000388       ??_C@_07FBLHGNAH@app?4exe?$AA@ 00011388     wince_unittests.obj
 0001:00000414       init                       00011414 f   gles1test1.obj
 0001:0000055c       display                    0001155c f   gles1test1.obj
 0001:00000678       main                       00011678 f   gles1test1.obj
 0001:00000960       WinMain                    00011960 f   wince_unittests.obj
 0001:00000b88       glTexParameterf            00011b88 f   libGLES_CM:libGLES_CM.dll
 0001:00000b98       glTexImage2D               00011b98 f   libGLES_CM:libGLES_CM.dll
 0001:00000ba8       glTexCoordPointer          00011ba8 f   libGLES_CM:libGLES_CM.dll
 0001:00000bb8       glColorPointer             00011bb8 f   libGLES_CM:libGLES_CM.dll
 0001:00000bc8       glVertexPointer            00011bc8 f   libGLES_CM:libGLES_CM.dll
 0001:00000bd8       glEnableClientState        00011bd8 f   libGLES_CM:libGLES_CM.dll
 0001:00000be8       glShadeModel               00011be8 f   libGLES_CM:libGLES_CM.dll
 0001:00000bf8       glClearColor               00011bf8 f   libGLES_CM:libGLES_CM.dll
 0001:00000c08       glDisable                  00011c08 f   libGLES_CM:libGLES_CM.dll
 0001:00000c18       glDrawArrays               00011c18 f   libGLES_CM:libGLES_CM.dll
 0001:00000c28       glEnable                   00011c28 f   libGLES_CM:libGLES_CM.dll
 0001:00000c38       glRotatef                  00011c38 f   libGLES_CM:libGLES_CM.dll
 0001:00000c48       glTranslatef               00011c48 f   libGLES_CM:libGLES_CM.dll
 0001:00000c58       glLoadIdentity             00011c58 f   libGLES_CM:libGLES_CM.dll
 0001:00000c68       glMatrixMode               00011c68 f   libGLES_CM:libGLES_CM.dll
 0001:00000c78       glClear                    00011c78 f   libGLES_CM:libGLES_CM.dll
 0001:00000c88       ReleasePowerRequirement    00011c88 f   coredll:COREDLL.dll
 0001:00000c98       NKDbgPrintfW               00011c98 f   coredll:COREDLL.dll
 0001:00000ca8       FormatMessageW             00011ca8 f   coredll:COREDLL.dll
 0001:00000cb8       GetLastError               00011cb8 f   coredll:COREDLL.dll
 0001:00000cc8       SetPowerRequirement        00011cc8 f   coredll:COREDLL.dll
 0001:00000cd8       WideCharToMultiByte        00011cd8 f   coredll:COREDLL.dll
 0001:00000d68       WinMainCRTStartup          00011d68 f   corelib0:pegwmain.obj
 0001:00000e64       exit                       00011e64 f   corelib0:cexit.obj
 0001:00000e7c       _exit                      00011e7c f   corelib0:cexit.obj
 0001:00000ebc       _initterm                  00011ebc f   corelib0:crt0dat.obj
 0001:00000ef0       _cinit                     00011ef0 f   corelib0:crt0dat.obj
 0001:00000f24       __security_init_cookie     00011f24 f   corelib0:seccinit.obj
 0001:00000f80       fprintf                    00011f80 f   corelib1:COREDLL.dll
 0001:00000f90       _getstdfilex               00011f90 f   corelib1:COREDLL.dll
 0001:00000fa0       atol                       00011fa0 f   corelib1:COREDLL.dll
 0001:00000fb0       _stricmp                   00011fb0 f   corelib1:COREDLL.dll
 0001:00000fc0       _isctype                   00011fc0 f   corelib1:COREDLL.dll
 0001:00000fd0       malloc                     00011fd0 f   corelib1:COREDLL.dll
 0001:00000fe0       wcslen                     00011fe0 f   corelib1:COREDLL.dll
 0001:00000ff0       memset                     00011ff0 f   corelib1:COREDLL.dll
 0001:00001000       _XcptFilter                00012000 f   corelib1:COREDLL.dll
 0001:00001010       __C_specific_handler       00012010 f   corelib1:COREDLL.dll
 0001:00001020       free                       00012020 f   corelib1:COREDLL.dll
 0001:00001030       __security_gen_cookie2     00012030 f   corelib1:COREDLL.dll
 0001:00001040       TerminateProcess           00012040 f   coredll:COREDLL.dll
 0001:00001064       __IMPORT_DESCRIPTOR_libGLES_CM 00012064     libGLES_CM:libGLES_CM.dll
 0001:00001078       __IMPORT_DESCRIPTOR_COREDLL 00012078     coredll:COREDLL.dll
 0001:0000108c       __NULL_IMPORT_DESCRIPTOR   0001208c     libGLES_CM:libGLES_CM.dll
 0002:00000000       __imp_TerminateProcess     00013000     coredll:COREDLL.dll
 0002:00000004       __imp___security_gen_cookie2 00013004     corelib1:COREDLL.dll
 0002:00000008       __imp_free                 00013008     corelib1:COREDLL.dll
 0002:0000000c       __imp___C_specific_handler 0001300c     corelib1:COREDLL.dll
 0002:00000010       __imp__XcptFilter          00013010     corelib1:COREDLL.dll
 0002:00000014       __imp_memset               00013014     corelib1:COREDLL.dll
 0002:00000018       __imp_wcslen               00013018     corelib1:COREDLL.dll
 0002:0000001c       __imp_malloc               0001301c     corelib1:COREDLL.dll
 0002:00000020       __imp__isctype             00013020     corelib1:COREDLL.dll
 0002:00000024       __imp__stricmp             00013024     corelib1:COREDLL.dll
 0002:00000028       __imp_atol                 00013028     corelib1:COREDLL.dll
 0002:0000002c       __imp___muls               0001302c     corelib1:COREDLL.dll
 0002:00000030       __imp___itos               00013030     corelib1:COREDLL.dll
 0002:00000034       __imp__getstdfilex         00013034     corelib1:COREDLL.dll
 0002:00000038       __imp_fprintf              00013038     corelib1:COREDLL.dll
 0002:0000003c       __imp_WideCharToMultiByte  0001303c     coredll:COREDLL.dll
 0002:00000040       __imp_SetPowerRequirement  00013040     coredll:COREDLL.dll
 0002:00000044       __imp_GetLastError         00013044     coredll:COREDLL.dll
 0002:00000048       __imp_FormatMessageW       00013048     coredll:COREDLL.dll
 0002:0000004c       __imp_NKDbgPrintfW         0001304c     coredll:COREDLL.dll
 0002:00000050       __imp_ReleasePowerRequirement 00013050     coredll:COREDLL.dll
 0002:00000054       \177COREDLL_NULL_THUNK_DATA 00013054     coredll:COREDLL.dll
 0002:00000058       __imp_eglCreateWindowSurface 00013058     libGLES_CM:libGLES_CM.dll
 0002:0000005c       __imp_eglChooseConfig      0001305c     libGLES_CM:libGLES_CM.dll
 0002:00000060       __imp_eglCreateContext     00013060     libGLES_CM:libGLES_CM.dll
 0002:00000064       __imp_eglGetDisplay        00013064     libGLES_CM:libGLES_CM.dll
 0002:00000068       __imp_eglInitialize        00013068     libGLES_CM:libGLES_CM.dll
 0002:0000006c       __imp_eglMakeCurrent       0001306c     libGLES_CM:libGLES_CM.dll
 0002:00000070       __imp_eglSwapInterval      00013070     libGLES_CM:libGLES_CM.dll
 0002:00000074       __imp_eglSwapBuffers       00013074     libGLES_CM:libGLES_CM.dll
 0002:00000078       __imp_eglTerminate         00013078     libGLES_CM:libGLES_CM.dll
 0002:0000007c       __imp_eglDestroySurface    0001307c     libGLES_CM:libGLES_CM.dll
 0002:00000080       __imp_eglDestroyContext    00013080     libGLES_CM:libGLES_CM.dll
 0002:00000084       __imp_glClear              00013084     libGLES_CM:libGLES_CM.dll
 0002:00000088       __imp_glMatrixMode         00013088     libGLES_CM:libGLES_CM.dll
 0002:0000008c       __imp_glLoadIdentity       0001308c     libGLES_CM:libGLES_CM.dll
 0002:00000090       __imp_glTranslatef         00013090     libGLES_CM:libGLES_CM.dll
 0002:00000094       __imp_glRotatef            00013094     libGLES_CM:libGLES_CM.dll
 0002:00000098       __imp_glEnable             00013098     libGLES_CM:libGLES_CM.dll
 0002:0000009c       __imp_glDrawArrays         0001309c     libGLES_CM:libGLES_CM.dll
 0002:000000a0       __imp_glDisable            000130a0     libGLES_CM:libGLES_CM.dll
 0002:000000a4       __imp_glClearColor         000130a4     libGLES_CM:libGLES_CM.dll
 0002:000000a8       __imp_glShadeModel         000130a8     libGLES_CM:libGLES_CM.dll
 0002:000000ac       __imp_glEnableClientState  000130ac     libGLES_CM:libGLES_CM.dll
 0002:000000b0       __imp_glVertexPointer      000130b0     libGLES_CM:libGLES_CM.dll
 0002:000000b4       __imp_glColorPointer       000130b4     libGLES_CM:libGLES_CM.dll
 0002:000000b8       __imp_glTexCoordPointer    000130b8     libGLES_CM:libGLES_CM.dll
 0002:000000bc       __imp_glTexImage2D         000130bc     libGLES_CM:libGLES_CM.dll
 0002:000000c0       __imp_glTexParameterf      000130c0     libGLES_CM:libGLES_CM.dll
 0002:000000c4       __imp_eglGetConfigs        000130c4     libGLES_CM:libGLES_CM.dll
 0002:000000c8       __imp_eglGetError          000130c8     libGLES_CM:libGLES_CM.dll
 0002:000000cc       \177libGLES_CM_NULL_THUNK_DATA 000130cc     libGLES_CM:libGLES_CM.dll
 0002:00000190       gui32WindowWidth           00013190     wince_unittests.obj
 0002:00000194       gui32WindowHeight          00013194     wince_unittests.obj
 0002:00000198       gui32PosX                  00013198     wince_unittests.obj
 0002:0000019c       gui32PosY                  0001319c     wince_unittests.obj
 0002:000001a0       __security_cookie          000131a0     corelib0:seccinit.obj
 0002:000001a4       __security_cookie_complement 000131a4     corelib0:seccinit.obj
 0002:000041ac       gbWindow                   000171ac     wince_unittests.obj
 0002:000041b0       ghWnd                      000171b0     wince_unittests.obj
 0002:000041b4       pfnRegisteredWndProc       000171b4     wince_unittests.obj
 0002:000041b8       _exitflag                  000171b8     corelib0:cexit.obj
 0002:000041bc       __onexitend                000171bc     <common>
 0002:000041c0       __onexitbegin              000171c0     <common>

 entry point at        0001:00000d68

 Static symbols

 0001:000003b8       handle_egl_error           000113b8 f   gles1test1.obj
 0001:00000cf0       WinMainCRTStartupHelper    00011cf0 f   corelib0:pegwmain.obj
 0001:00000d9c       doexit                     00011d9c f   corelib0:cexit.obj
